******************************************************************************
             TMS320C2000 Linker PC v22.6.0                     
******************************************************************************
>> Linked Thu Apr 20 08:24:33 2023

OUTPUT FILE NAME:   <led_ex1_c28x_cm_blinky_cpu1.out>
ENTRY POINT SYMBOL: "code_start"  address: 00080000


MEMORY CONFIGURATION

         name            origin    length      used     unused   attr    fill
----------------------  --------  ---------  --------  --------  ----  --------
  BOOT_RSVD             00000002   000001af  00000000  000001af  RWIX
  RAMM0                 000001b1   0000024f  00000000  0000024f  RWIX
  RAMM1                 00000400   000003f8  00000100  000002f8  RWIX
  RAMLS0                00008000   00000800  00000122  000006de  RWIX
  RAMLS1                00008800   00000800  00000000  00000800  RWIX
  RAMLS2                00009000   00000800  00000000  00000800  RWIX
  RAMLS3                00009800   00000800  00000000  00000800  RWIX
  RAMLS4                0000a000   00000800  00000000  00000800  RWIX
  RAMLS5                0000a800   00000800  0000000a  000007f6  RWIX
  RAMLS6                0000b000   00000800  00000000  00000800  RWIX
  RAMLS7                0000b800   00000800  00000000  00000800  RWIX
  RAMD0                 0000c000   00000800  00000000  00000800  RWIX
  RAMD1                 0000c800   00000800  00000000  00000800  RWIX
  RAMGS0                0000d000   00001000  00000000  00001000  RWIX
  RAMGS1                0000e000   00001000  00000000  00001000  RWIX
  RAMGS2                0000f000   00001000  00000000  00001000  RWIX
  RAMGS3                00010000   00001000  00000000  00001000  RWIX
  RAMGS4                00011000   00001000  00000000  00001000  RWIX
  RAMGS5                00012000   00001000  00000000  00001000  RWIX
  RAMGS6                00013000   00001000  00000000  00001000  RWIX
  RAMGS7                00014000   00001000  00000000  00001000  RWIX
  RAMGS8                00015000   00001000  00000000  00001000  RWIX
  RAMGS9                00016000   00001000  00000000  00001000  RWIX
  RAMGS10               00017000   00001000  00000000  00001000  RWIX
  RAMGS11               00018000   00001000  00000000  00001000  RWIX
  RAMGS12               00019000   00001000  00000000  00001000  RWIX
  RAMGS13               0001a000   00001000  00000000  00001000  RWIX
  RAMGS14               0001b000   00001000  00000000  00001000  RWIX
  RAMGS15               0001c000   00000ff8  00000000  00000ff8  RWIX
  CMTOCPURAM            00038000   00000800  00000088  00000778  RWIX
  CPUTOCMRAM            00039000   00000800  00000088  00000778  RWIX
  CPU1TOCPU2RAM         0003a000   00000800  00000088  00000778  RWIX
  CPU2TOCPU1RAM         0003b000   00000800  00000088  00000778  RWIX
  CANA_MSG_RAM          00049000   00000800  00000000  00000800  RWIX
  CANB_MSG_RAM          0004b000   00000800  00000000  00000800  RWIX
  BEGIN                 00080000   00000002  00000002  00000000  RWIX
  FLASH0                00080002   00001ffe  00000000  00001ffe  RWIX
  FLASH1                00082000   00002000  00000fba  00001046  RWIX
  FLASH2                00084000   00002000  00000000  00002000  RWIX
  FLASH3                00086000   00002000  00000122  00001ede  RWIX
  FLASH4                00088000   00008000  00000014  00007fec  RWIX
  FLASH5                00090000   00008000  0000037d  00007c83  RWIX
  FLASH6                00098000   00008000  00000000  00008000  RWIX
  FLASH7                000a0000   00008000  00000000  00008000  RWIX
  FLASH8                000a8000   00008000  00000000  00008000  RWIX
  FLASH9                000b0000   00008000  00000000  00008000  RWIX
  FLASH10               000b8000   00002000  00000000  00002000  RWIX
  FLASH11               000ba000   00002000  00000000  00002000  RWIX
  FLASH12               000bc000   00002000  00000000  00002000  RWIX
  FLASH13               000be000   00001ff0  00000000  00001ff0  RWIX
  RESET                 003fffc0   00000002  00000000  00000002  RWIX


SECTION ALLOCATION MAP

 output                                  attributes/
section   page    origin      length       input sections
--------  ----  ----------  ----------   ----------------
codestart 
*          0    00080000    00000002     
                  00080000    00000002     f2838x_codestartbranch.obj (codestart)

.cinit     0    00088000    00000014     
                  00088000    00000009     (.cinit..data.load) [load image, compression = lzss]
                  00088009    00000001     --HOLE-- [fill = 0]
                  0008800a    00000004     (__TI_handler_table)
                  0008800e    00000002     --HOLE-- [fill = 0]
                  00088010    00000004     (__TI_cinit_table)

.reset     0    003fffc0    00000000     DSECT

.stack     0    00000400    00000100     UNINITIALIZED
                  00000400    00000100     --HOLE--

.init_array 
*          0    00082000    00000000     UNINITIALIZED

.data      0    0000a800    0000000a     UNINITIALIZED
                  0000a800    00000006     rts2800_fpu64_eabi.lib : exit.c.obj (.data)
                  0000a806    00000002                            : _lock.c.obj (.data:_lock)
                  0000a808    00000002                            : _lock.c.obj (.data:_unlock)

MSGRAM_CM_TO_CPU 
*          0    00038000    00000088     UNINITIALIZED
                  00038000    00000088     driverlib.lib : ipc.obj (MSGRAM_CM_TO_CPU)

MSGRAM_CPU_TO_CM 
*          0    00039000    00000088     UNINITIALIZED
                  00039000    00000088     driverlib.lib : ipc.obj (MSGRAM_CPU_TO_CM)

.const     0    00090000    0000037d     
                  00090000    00000098     driverlib.lib : flash.obj (.const:.string)
                  00090098    00000097                   : gpio.obj (.const:.string)
                  0009012f    00000001     --HOLE-- [fill = 0]
                  00090130    00000097                   : sysctl.obj (.const:.string)
                  000901c7    00000001     --HOLE-- [fill = 0]
                  000901c8    00000094                   : dcc.obj (.const:.string)
                  0009025c    00000088                   : ipc.obj (.const:IPC_Instance)
                  000902e4    00000055     device.obj (.const:.string)
                  00090339    00000001     --HOLE-- [fill = 0]
                  0009033a    00000043     led_ex1_c28x_cm_blinky_cpu1.obj (.const:.string)

MSGRAM_CPU1_TO_CPU2 
*          0    0003a000    00000088     UNINITIALIZED
                  0003a000    00000088     driverlib.lib : ipc.obj (MSGRAM_CPU1_TO_CPU2)

MSGRAM_CPU2_TO_CPU1 
*          0    0003b000    00000088     UNINITIALIZED
                  0003b000    00000088     driverlib.lib : ipc.obj (MSGRAM_CPU2_TO_CPU1)

.TI.ramfunc 
*          0    00086000    00000122     RUN ADDR = 00008000
                  00086000    0000003f     driverlib.lib : flash.obj (.TI.ramfunc:Flash_initModule)
                  0008603f    0000002c                   : flash.obj (.TI.ramfunc:Flash_setBankPowerMode)
                  0008606b    00000022                   : flash.obj (.TI.ramfunc:Flash_setWaitstates)
                  0008608d    0000001d                   : flash.obj (.TI.ramfunc:Flash_setPumpPowerMode)
                  000860aa    00000018                   : flash.obj (.TI.ramfunc:Flash_disableCache)
                  000860c2    00000018                   : flash.obj (.TI.ramfunc:Flash_disablePrefetch)
                  000860da    00000017                   : flash.obj (.TI.ramfunc:Flash_enableCache)
                  000860f1    00000017                   : flash.obj (.TI.ramfunc:Flash_enablePrefetch)
                  00086108    00000016                   : flash.obj (.TI.ramfunc:Flash_enableECC)
                  0008611e    00000004                   : sysctl.obj (.TI.ramfunc)

.text      0    00082000    00000fba     
                  00082000    00000167     device.obj (.text:Device_enableAllPeripherals)
                  00082167    00000132     driverlib.lib : sysctl.obj (.text:SysCtl_setClock)
                  00082299    00000118                   : sysctl.obj (.text:SysCtl_isPLLValid)
                  000823b1    00000113                   : sysctl.obj (.text:SysCtl_setAuxClock)
                  000824c4    000000ca                   : dcc.obj (.text:DCC_verifyClockFrequency)
                  0008258e    00000088     rts2800_fpu64_eabi.lib : fs_div28.asm.obj (.text)
                  00082616    00000073     driverlib.lib : dcc.obj (.text:DCC_setCounterSeeds)
                  00082689    00000073                   : sysctl.obj (.text:DCC_setCounterSeeds)
                  000826fc    0000006b     device.obj (.text:Device_init)
                  00082767    00000061     driverlib.lib : sysctl.obj (.text:SysCtl_getAuxClock)
                  000827c8    00000060                   : sysctl.obj (.text:SysCtl_getClock)
                  00082828    00000052                   : gpio.obj (.text:GPIO_setPadConfig)
                  0008287a    00000047                   : sysctl.obj (.text:SysCtl_selectOscSourceAuxPLL)
                  000828c1    00000044     led_ex1_c28x_cm_blinky_cpu1.obj (.text:GPIO_writePin)
                  00082905    00000042     driverlib.lib : sysctl.obj (.text:SysCtl_selectOscSource)
                  00082947    0000003d                   : interrupt.obj (.text:Interrupt_initModule)
                  00082984    0000003c     led_ex1_c28x_cm_blinky_cpu1.obj (.text:main)
                  000829c0    00000037     driverlib.lib : gpio.obj (.text:GPIO_setMasterCore)
                  000829f7    00000031                   : gpio.obj (.text:GPIO_setDirectionMode)
                  00082a28    0000002e     rts2800_fpu64_eabi.lib : copy_decompress_lzss.c.obj (.text:decompress:lzss)
                  00082a56    0000002b                            : autoinit.c.obj (.text:__TI_auto_init_nobinit_nopinit)
                  00082a81    00000029                            : exit.c.obj (.text)
                  00082aaa    00000027     driverlib.lib : sysctl.obj (.text:SysCtl_pollX1Counter)
                  00082ad1    00000025                   : sysctl.obj (.text:SysCtl_controlCMReset)
                  00082af6    00000024                   : dcc.obj (.text:DCC_enableSingleShotMode)
                  00082b1a    00000024                   : sysctl.obj (.text:DCC_enableSingleShotMode)
                  00082b3e    00000024                   : sysctl.obj (.text:SysCtl_selectXTAL)
                  00082b62    00000021     device.obj (.text:Device_initGPIO)
                  00082b83    0000001e     driverlib.lib : dcc.obj (.text:DCC_setCounter0ClkSource)
                  00082ba1    0000001e                   : sysctl.obj (.text:DCC_setCounter0ClkSource)
                  00082bbf    0000001e                   : dcc.obj (.text:DCC_setCounter1ClkSource)
                  00082bdd    0000001e                   : sysctl.obj (.text:DCC_setCounter1ClkSource)
                  00082bfb    0000001e     device.obj (.text:Device_verifyXTAL)
                  00082c19    0000001e     driverlib.lib : interrupt.obj (.text:Interrupt_initVectorTable)
                  00082c37    0000001d     rts2800_fpu64_eabi.lib : memcpy.c.obj (.text)
                  00082c54    0000001c     driverlib.lib : dcc.obj (.text:DCC_getErrorStatus)
                  00082c70    0000001c                   : dcc.obj (.text:DCC_getSingleShotStatus)
                  00082c8c    0000001a                   : dcc.obj (.text:DCC_isBaseValid)
                  00082ca6    0000001a                   : sysctl.obj (.text:DCC_isBaseValid)
                  00082cc0    0000001a                   : sysctl.obj (.text:SysCtl_getLowSpeedClock)
                  00082cda    0000001a                   : sysctl.obj (.text:SysCtl_selectXTALSingleEnded)
                  00082cf4    00000019     device.obj (.text:IPC_setBootMode)
                  00082d0d    00000019     rts2800_fpu64_eabi.lib : boot28.asm.obj (.text)
                  00082d26    00000017     device.obj (.text:SysCtl_enablePeripheral)
                  00082d3d    00000017     driverlib.lib : sysctl.obj (.text:SysCtl_enablePeripheral)
                  00082d54    00000016                   : dcc.obj (.text:DCC_disableDoneSignal)
                  00082d6a    00000016                   : sysctl.obj (.text:DCC_disableDoneSignal)
                  00082d80    00000016                   : dcc.obj (.text:DCC_enableDoneSignal)
                  00082d96    00000016     device.obj (.text:Device_bootCM)
                  00082dac    00000015     driverlib.lib : dcc.obj (.text:DCC_clearDoneFlag)
                  00082dc1    00000015                   : sysctl.obj (.text:DCC_clearDoneFlag)
                  00082dd6    00000015                   : dcc.obj (.text:DCC_clearErrorFlag)
                  00082deb    00000015                   : sysctl.obj (.text:DCC_clearErrorFlag)
                  00082e00    00000015                   : dcc.obj (.text:DCC_disableErrorSignal)
                  00082e15    00000015                   : sysctl.obj (.text:DCC_disableErrorSignal)
                  00082e2a    00000015     device.obj (.text:GPIO_unlockPortConfig)
                  00082e3f    00000014     driverlib.lib : dcc.obj (.text:DCC_disableModule)
                  00082e53    00000014                   : sysctl.obj (.text:DCC_disableModule)
                  00082e67    00000014                   : dcc.obj (.text:DCC_enableErrorSignal)
                  00082e7b    00000014                   : dcc.obj (.text:DCC_enableModule)
                  00082e8f    00000014                   : sysctl.obj (.text:DCC_enableModule)
                  00082ea3    00000013     device.obj (.text:Device_enableUnbondedGPIOPullupsFor176Pin)
                  00082eb6    00000011     device.obj (.text:Device_enableUnbondedGPIOPullups)
                  00082ec7    00000011     device.obj (.text:SysCtl_setCMClk)
                  00082ed8    00000010     driverlib.lib : flash.obj (.text:Flash_isCtrlBaseValid)
                  00082ee8    00000010                   : flash.obj (.text:Flash_isECCBaseValid)
                  00082ef8    0000000f     device.obj (.text:IPC_setFlagLtoR)
                  00082f07    0000000e     driverlib.lib : gpio.obj (.text:GPIO_isPinValid)
                  00082f15    0000000e     led_ex1_c28x_cm_blinky_cpu1.obj (.text:GPIO_isPinValid)
                  00082f23    0000000e     driverlib.lib : interrupt.obj (.text:Interrupt_defaultHandler)
                  00082f31    0000000d                   : interrupt.obj (.text:Interrupt_disableMaster)
                  00082f3e    0000000d     device.obj (.text:SysCtl_setLowSpeedClock)
                  00082f4b    0000000c     driverlib.lib : sysctl.obj (.text:SysCtl_setPLLSysClk)
                  00082f57    0000000c     rts2800_fpu64_eabi.lib : args_main.c.obj (.text)
                  00082f63    0000000b     device.obj (.text:SysCtl_isCMReset)
                  00082f6e    0000000b     driverlib.lib : sysctl.obj (.text:SysCtl_isCMReset)
                  00082f79    0000000b                   : sysctl.obj (.text:SysCtl_isMCDClockFailureDetected)
                  00082f84    00000009     rts2800_fpu64_eabi.lib : _lock.c.obj (.text)
                  00082f8d    00000008     device.obj (.text:SysCtl_disableWatchdog)
                  00082f95    00000008     rts2800_fpu64_eabi.lib : copy_decompress_none.c.obj (.text:decompress:none)
                  00082f9d    00000008     f2838x_codestartbranch.obj (.text)
                  00082fa5    00000007     driverlib.lib : sysctl.obj (.text:SysCtl_resetMCD)
                  00082fac    00000007     device.obj (.text:__error__)
                  00082fb3    00000002     driverlib.lib : interrupt.obj (.text:Interrupt_illegalOperationHandler)
                  00082fb5    00000002                   : interrupt.obj (.text:Interrupt_nmiHandler)
                  00082fb7    00000002     rts2800_fpu64_eabi.lib : pre_init.c.obj (.text)
                  00082fb9    00000001                            : startup.c.obj (.text)

MODULE SUMMARY

       Module                            code   ro data   rw data
       ------                            ----   -------   -------
    .\
       led_ex1_c28x_cm_blinky_cpu1.obj   142    67        0      
    +--+---------------------------------+------+---------+---------+
       Total:                            142    67        0      
                                                                 
    .\device\
       device.obj                        727    85        0      
       f2838x_codestartbranch.obj        10     0         0      
    +--+---------------------------------+------+---------+---------+
       Total:                            737    85        0      
                                                                 
    C:/ti/c2000/C2000Ware_4_02_00_00/driverlib/f2838x/driverlib/ccs/Debug/driverlib.lib
       sysctl.obj                        1789   151       0      
       dcc.obj                           662    148       0      
       flash.obj                         604    152       0      
       ipc.obj                           0      136       544    
       gpio.obj                          200    151       0      
       interrupt.obj                     122    0         0      
    +--+---------------------------------+------+---------+---------+
       Total:                            3377   738       544    
                                                                 
    C:\ti\ccs1210\ccs\tools\compiler\ti-cgt-c2000_22.6.0.LTS\lib\rts2800_fpu64_eabi.lib
       fs_div28.asm.obj                  136    0         0      
       exit.c.obj                        41     0         6      
       copy_decompress_lzss.c.obj        46     0         0      
       autoinit.c.obj                    43     0         0      
       memcpy.c.obj                      29     0         0      
       boot28.asm.obj                    25     0         0      
       _lock.c.obj                       9      0         4      
       args_main.c.obj                   12     0         0      
       copy_decompress_none.c.obj        8      0         0      
       pre_init.c.obj                    2      0         0      
       startup.c.obj                     1      0         0      
    +--+---------------------------------+------+---------+---------+
       Total:                            352    0         10     
                                                                 
       Stack:                            0      0         256    
       Linker Generated:                 0      17        0      
    +--+---------------------------------+------+---------+---------+
       Grand Total:                      4608   907       810    


LINKER GENERATED COPY TABLES

__TI_cinit_table @ 00088010 records: 1, size/record: 4, table size: 4
	.data: load addr=00088000, load size=00000009 bytes, run addr=0000a800, run size=0000000a bytes, compression=lzss


LINKER GENERATED HANDLER TABLE

__TI_handler_table @ 0008800a records: 2, size/record: 2, table size: 4
	index: 0, handler: __TI_decompress_lzss
	index: 1, handler: __TI_decompress_none


GLOBAL DATA SYMBOLS: SORTED BY DATA PAGE

address     data page           name
--------    ----------------    ----
00000400      10 (00000400)     __stack

0000a800     2a0 (0000a800)     __TI_enable_exit_profile_output
0000a802     2a0 (0000a800)     __TI_cleanup_ptr
0000a804     2a0 (0000a800)     __TI_dtors_ptr
0000a806     2a0 (0000a800)     _lock
0000a808     2a0 (0000a800)     _unlock

00038000     e00 (00038000)     IPC_CPU_To_CM_GetBuffer

00039000     e40 (00039000)     IPC_CPU_To_CM_PutBuffer

0003a000     e80 (0003a000)     IPC_CPU1_To_CPU2_PutBuffer

0003b000     ec0 (0003b000)     IPC_CPU1_To_CPU2_GetBuffer

0009025c    2409 (00090240)     IPC_Instance


GLOBAL SYMBOLS: SORTED ALPHABETICALLY BY Name 

page  address   name                                     
----  -------   ----                                     
0     00082a81  C$$EXIT                                  
0     000824c4  DCC_verifyClockFrequency                 
0     00082d96  Device_bootCM                            
0     00082000  Device_enableAllPeripherals              
0     00082eb6  Device_enableUnbondedGPIOPullups         
0     00082ea3  Device_enableUnbondedGPIOPullupsFor176Pin
0     000826fc  Device_init                              
0     00082b62  Device_initGPIO                          
0     00082bfb  Device_verifyXTAL                        
0     00008000  Flash_initModule                         
0     000829f7  GPIO_setDirectionMode                    
0     000829c0  GPIO_setMasterCore                       
0     00082828  GPIO_setPadConfig                        
0     0003b000  IPC_CPU1_To_CPU2_GetBuffer               
0     0003a000  IPC_CPU1_To_CPU2_PutBuffer               
0     00038000  IPC_CPU_To_CM_GetBuffer                  
0     00039000  IPC_CPU_To_CM_PutBuffer                  
0     0009025c  IPC_Instance                             
0     00082947  Interrupt_initModule                     
0     00082c19  Interrupt_initVectorTable                
0     00086122  RamfuncsLoadEnd                          
abs   00000122  RamfuncsLoadSize                         
0     00086000  RamfuncsLoadStart                        
0     00008122  RamfuncsRunEnd                           
abs   00000122  RamfuncsRunSize                          
0     00008000  RamfuncsRunStart                         
0     00082ad1  SysCtl_controlCMReset                    
0     0000811e  SysCtl_delay                             
0     00082767  SysCtl_getAuxClock                       
0     000827c8  SysCtl_getClock                          
0     00082cc0  SysCtl_getLowSpeedClock                  
0     00082299  SysCtl_isPLLValid                        
0     00082905  SysCtl_selectOscSource                   
0     0008287a  SysCtl_selectOscSourceAuxPLL             
0     00082b3e  SysCtl_selectXTAL                        
0     00082cda  SysCtl_selectXTALSingleEnded             
0     000823b1  SysCtl_setAuxClock                       
0     00082167  SysCtl_setClock                          
0     00088010  __TI_CINIT_Base                          
0     00088014  __TI_CINIT_Limit                         
0     00088014  __TI_CINIT_Warm                          
0     0008800a  __TI_Handler_Table_Base                  
0     0008800e  __TI_Handler_Table_Limit                 
0     00000500  __TI_STACK_END                           
abs   00000100  __TI_STACK_SIZE                          
0     00082a56  __TI_auto_init_nobinit_nopinit           
0     0000a802  __TI_cleanup_ptr                         
0     00082a28  __TI_decompress_lzss                     
0     00082f95  __TI_decompress_none                     
0     0000a804  __TI_dtors_ptr                           
0     0000a800  __TI_enable_exit_profile_output          
abs   ffffffff  __TI_pprof_out_hndl                      
abs   ffffffff  __TI_prof_data_size                      
abs   ffffffff  __TI_prof_data_start                     
0     0008258e  __c28xabi_divf                           
n/a   UNDEFED   __c_args__                               
0     00082fac  __error__                                
0     00000400  __stack                                  
0     00082f57  _args_main                               
0     00082d0d  _c_int00                                 
0     0000a806  _lock                                    
0     00082f8c  _nop                                     
0     00082f88  _register_lock                           
0     00082f84  _register_unlock                         
0     00082fb9  _system_post_cinit                       
0     00082fb7  _system_pre_init                         
0     0000a808  _unlock                                  
0     00082a81  abort                                    
0     00080000  code_start                               
0     00082a83  exit                                     
0     00082984  main                                     
0     00082c37  memcpy                                   


GLOBAL SYMBOLS: SORTED BY Symbol Address 

page  address   name                                     
----  -------   ----                                     
0     00000400  __stack                                  
0     00000500  __TI_STACK_END                           
0     00008000  Flash_initModule                         
0     00008000  RamfuncsRunStart                         
0     0000811e  SysCtl_delay                             
0     00008122  RamfuncsRunEnd                           
0     0000a800  __TI_enable_exit_profile_output          
0     0000a802  __TI_cleanup_ptr                         
0     0000a804  __TI_dtors_ptr                           
0     0000a806  _lock                                    
0     0000a808  _unlock                                  
0     00038000  IPC_CPU_To_CM_GetBuffer                  
0     00039000  IPC_CPU_To_CM_PutBuffer                  
0     0003a000  IPC_CPU1_To_CPU2_PutBuffer               
0     0003b000  IPC_CPU1_To_CPU2_GetBuffer               
0     00080000  code_start                               
0     00082000  Device_enableAllPeripherals              
0     00082167  SysCtl_setClock                          
0     00082299  SysCtl_isPLLValid                        
0     000823b1  SysCtl_setAuxClock                       
0     000824c4  DCC_verifyClockFrequency                 
0     0008258e  __c28xabi_divf                           
0     000826fc  Device_init                              
0     00082767  SysCtl_getAuxClock                       
0     000827c8  SysCtl_getClock                          
0     00082828  GPIO_setPadConfig                        
0     0008287a  SysCtl_selectOscSourceAuxPLL             
0     00082905  SysCtl_selectOscSource                   
0     00082947  Interrupt_initModule                     
0     00082984  main                                     
0     000829c0  GPIO_setMasterCore                       
0     000829f7  GPIO_setDirectionMode                    
0     00082a28  __TI_decompress_lzss                     
0     00082a56  __TI_auto_init_nobinit_nopinit           
0     00082a81  C$$EXIT                                  
0     00082a81  abort                                    
0     00082a83  exit                                     
0     00082ad1  SysCtl_controlCMReset                    
0     00082b3e  SysCtl_selectXTAL                        
0     00082b62  Device_initGPIO                          
0     00082bfb  Device_verifyXTAL                        
0     00082c19  Interrupt_initVectorTable                
0     00082c37  memcpy                                   
0     00082cc0  SysCtl_getLowSpeedClock                  
0     00082cda  SysCtl_selectXTALSingleEnded             
0     00082d0d  _c_int00                                 
0     00082d96  Device_bootCM                            
0     00082ea3  Device_enableUnbondedGPIOPullupsFor176Pin
0     00082eb6  Device_enableUnbondedGPIOPullups         
0     00082f57  _args_main                               
0     00082f84  _register_unlock                         
0     00082f88  _register_lock                           
0     00082f8c  _nop                                     
0     00082f95  __TI_decompress_none                     
0     00082fac  __error__                                
0     00082fb7  _system_pre_init                         
0     00082fb9  _system_post_cinit                       
0     00086000  RamfuncsLoadStart                        
0     00086122  RamfuncsLoadEnd                          
0     0008800a  __TI_Handler_Table_Base                  
0     0008800e  __TI_Handler_Table_Limit                 
0     00088010  __TI_CINIT_Base                          
0     00088014  __TI_CINIT_Limit                         
0     00088014  __TI_CINIT_Warm                          
0     0009025c  IPC_Instance                             
abs   00000100  __TI_STACK_SIZE                          
abs   00000122  RamfuncsLoadSize                         
abs   00000122  RamfuncsRunSize                          
abs   ffffffff  __TI_pprof_out_hndl                      
abs   ffffffff  __TI_prof_data_size                      
abs   ffffffff  __TI_prof_data_start                     
n/a   UNDEFED   __c_args__                               

[72 symbols]
